:103800000C94241C0C943F1C0C943F1C0C943F1CE7
:103810000C943F1C0C943F1C0C943F1C0C943F1CBC
:103820000C943F1C0C943F1C0C943F1C0C943F1CAC
:103830000C943F1C0C943F1C0C943F1C0C943F1C9C
:103840000C943F1C0C943F1C11241FBECFE5D4E008
:10385000DEBFCDBF10E0A0E6B0E0EEEDFEE302C0BB
:1038600005900D92A036B107D9F711E0A0E6B0E0BF
:1038700001C01D92A43AB107E1F70C94321F0C94D9
:10388000001C0F92AF93BF93CF93DF93EF93FF93FF
:10389000FC01EA01DB01C895099231961197D9F72D
:1038A000FF91EF91DF91CF91BF91AF910F9008956C
:1038B0000F921F920F93AF93BF93CF93DF93EF932A
:1038C000FF93FC01EA01DB010990199001E043D06C
:1038D00032961297C9F7FC0103E03DD005E03BD0DA
:1038E000FF91EF91DF91CF91BF91AF910F911F9019
:1038F0000F9008950F931F93EF93FF93FC0103E044
:103900002AD000E810E0E00FF11FE617F707B9F73B
:10391000FF91EF911F910F9108950F930F9222D075
:10392000082E09E018D00F900F9108950F930F9271
:10393000EF93FF9317D0FC0160935700C895802D3B
:10394000FF91EF910F900F9108950F930BD001E12C
:1039500002D00F910895E199FECF00935700E895AA
:10396000FFFF00000091570000FDFCCF089583E0A9
:1039700089B98AB188618AB908958AB1877E8AB97E
:1039800008958CB95E9BFECF5E9A08958CB19927FD
:1039900008958BB19927807890700895EF92FF92E7
:1039A0000F931F93CF93DF937B01C0E0D0E0C61746
:1039B000D70770F48C010E94C91C8823E1F30E9490
:1039C000C61CF80181938F012196CE15DF0598F36F
:1039D00081E090E0DF91CF911F910F91FF90EF90E8
:1039E0000895EF92FF920F931F93CF93DF937C0183
:1039F0008B01C0E0D0E0C017D10738F4F701819106
:103A00007F010E94C11C2196F6CF81E090E0DF91FA
:103A1000CF911F910F91FF90EF90089540E050E0FB
:103A20004817590750F42AE633E00000215030408F
:103A300037FFFBCF4F5F5F4FF3CF08950E94BD1C50
:103A40000E94000008950E94C91C8823E1F30E948F
:103A5000C61C803219F481E090E0089585E10E944F
:103A6000C11C80E090E0089590E0282F3327213892
:103A7000310589F02238310524F42038310549F028
:103A80000DC02238310549F02839310539F493E069
:103A900005C092E003C091E001C092E1892F99270F
:103AA000089540E050E06091A0007091A100461799
:103AB0005707D0F42091A2013091A301E2EAF0E08F
:103AC0003FBB2EBB2F5F3F4F80818DBBE29AE19AB7
:103AD000E199FECF4F5F5F4F31964617570780F34E
:103AE0003093A3012093A201089540E050E060913B
:103AF000A0007091A10046175707B0F42091A201D1
:103B00003091A301E2EAF0E03FBB2EBB2F5F3F4FB5
:103B1000E09A8DB381934F5F5F4F46175707A0F32D
:103B20003093A3012093A2010895CF93DF93C0E0C7
:103B3000D0E08091A0009091A100C817D907A0F40F
:103B4000CE018E559F4F2091A2013091A301220FEB
:103B5000331FAC0160E870E0C9018C0F9D1F0E940B
:103B6000581CC058DF4FE5CF0E94A51CDF91CF91B4
:103B700008958091A2019091A30142EA50E06091E2
:103B8000A0007091A100880F991F0E94411C089508
:103B9000CF93C0E069E081E090E00E94961C9927F5
:103BA00084FF03C08F7E0E948D1C0E94C91C882345
:103BB000E1F30E94C61C9927823591051CF58035DA
:103BC00091050CF05CC08134910509F462C0823427
:103BD00091057CF481339105B1F18233910524F490
:103BE000C09709F44CC038C18034910509F438C13C
:103BF00033C18234910509F45FC08534910509F41D
:103C00005EC02AC18635910509F4F1C0873591055A
:103C10004CF48235910509F45FC08535910509F4AE
:103C200069C01AC18437910509F4A4C0853791058C
:103C30002CF48436910509F476C00EC185379105C0
:103C400009F4C5C009C10E94231D882309F4ADCF22
:103C500084E10E94C11C81E40E94C11C86E50E948F
:103C6000C11C82E50E94C11C80E20E94C11C83E548
:103C70000E94C11C84E50E94C11C8BE406C00E9406
:103C8000231D882309F491CF84E10E94C11C80E1A7
:103C9000E4C061E070E080E690E00E94CE1C0E94EB
:103CA000231D882309F481CF84E10E94C11C8091E7
:103CB00060000E94341DE9CF64E170E008C061E05B
:103CC00070E080E690E00E94CE1C64E070E080E648
:103CD00090E00E94CE1CD3CF0E94231D882309F4BC
:103CE00064CF60E070E480E090E00E947A1C0E9463
:103CF000A51CCACF62E070E080E690E00E94CE1C76
:103D00000E94231D882309F450CF209160008091E8
:103D100061009927982F8827820F911D9093A30106
:103D20008093A201B1CF63E070E080E690E00E9452
:103D3000CE1C20916100809160009927982F8827E0
:103D4000820F911D9093A1008093A000BC0182EA94
:103D500090E00E94CE1C0E94231D882309F425CFE9
:103D600080916200863419F40E94951D8DCF0E94C7
:103D7000511D8ACF63E070E080E690E00E94CE1C87
:103D800020916100809160009927982F8827820FE9
:103D9000911D9093A1008093A0000E94231D882371
:103DA00009F403CF80916200863419F40E94B91D92
:103DB00002C00E94751D84E10E94C11C6091A00098
:103DC0007091A10082EA90E00E94F11C60CF0E94F5
:103DD000231D882309F4E9CE84E10E94C11C8EE1F1
:103DE0000E94C11C84E90E94C11C82E04ECF64E0A5
:103DF00070E080E690E00E94CE1C0E94231D882384
:103E000009F4D3CE84E10E94C11C8091600080350A
:103E100031F480916100882361F4C82F17C0883580
:103E200031F480916100883061F4C3E00FC08035C7
:103E300031F480916100883049F4C2E007C08835D0
:103E400029F480916100882309F4C1E069E08C2F96
:103E500099270E94961C19CF85E10E94C11CA5CE0E
:103E6000CF910895CFE5D4E0DEBFCDBFCEE1F89489
:103E7000AEEFB1E00E94661F802D843B71F4AFEF7E
:103E8000B1E00E94661F802D833C39F4ADEFB1E0B4
:103E90000E94661F802D992781BF0E94B71C0E9437
:103EA000C61C84E690E00E940E1D0E94C91C882357
:103EB00019F00E94C81D04C0C150C8BBCC2389F7AB
:103EC0000E941E1D80E090E00C946E1FE199FECFD1
:0E3ED000BFBBAEBBE09A11960DB20895FFCFB6
:0400000300003800C1
:00000001FF
